******************************************************************************
               TMS320C6x Linker PC v7.4.1                      
******************************************************************************
>> Linked Mon Jun 17 09:45:57 2013

OUTPUT FILE NAME:   <Memory_Test.out>
ENTRY POINT SYMBOL: "_c_int00"  address: 008143c0


MEMORY CONFIGURATION

         name            origin    length      used     unused   attr    fill
----------------------  --------  ---------  --------  --------  ----  --------
  LL2                   00800000   00080000  0002124a  0005edb6  RWIX


SEGMENT ALLOCATION MAP

run origin  load origin   length   init length attrs members
----------  ----------- ---------- ----------- ----- -------
00800000    00800000    00014c68   00014c68    r-x
  00800000    00800000    00014c40   00014c40    r-x .text
  00814c40    00814c40    00000028   00000028    r-- .switch
00814c68    00814c68    00001000   00000000    rw-
  00814c68    00814c68    00001000   00000000    rw- .stack
00815c68    00815c68    00008a30   00008210    rw-
  00815c68    00815c68    00008210   00008210    rw- .far
  0081de78    0081de78    00000020   00000000    rw- .bss
  0081de98    0081de98    00000800   00000000    rw- .sysmem
0081e698    0081e698    00000484   00000484    rw-
  0081e698    0081e698    00000484   00000484    rw- .fardata
0081eb20    0081eb20    0000225e   0000225e    r--
  0081eb20    0081eb20    0000225e   0000225e    r-- .const
00820d80    00820d80    000000c4   000000c4    rw-
  00820d80    00820d80    000000c4   000000c4    rw- .neardata
00820e44    00820e44    000002e8   000002e8    r--
  00820e44    00820e44    000002e8   000002e8    r-- .cinit
0082112c    0082112c    00000120   00000000    rw-
  0082112c    0082112c    00000120   00000000    rw- .cio


SECTION ALLOCATION MAP

 output                                  attributes/
section   page    origin      length       input sections
--------  ----  ----------  ----------   ----------------
.text      0    00800000    00014c40     
                  00800000    00004ca0     KeyStone_common.obj (.text)
                  00804ca0    00002860     KeyStone_DDR_Init.obj (.text)
                  00807500    00000ba0     mem_test_main.obj (.text)
                  008080a0    00000a60     mem_test_DMA.obj (.text)
                  00808b00    00000940     rts6600_elf.lib : _scanfi.obj (.text:_scanfi)
                  00809440    000006c0     mem_test_DSP_core.obj (.text)
                  00809b00    000006a0     rts6600_elf.lib : _scanfi.obj (.text:_sset_arg)
                  0080a1a0    00000600     KeyStone_common.obj (.text:retain)
                  0080a7a0    000005c0     rts6600_elf.lib : divd.obj (.text:__c6xabi_divd)
                  0080ad60    000005c0                     : _printfi.obj (.text:_getarg_diouxp)
                  0080b320    00000520                     : strtod.obj (.text:strtod)
                  0080b840    00000520                     : strtold.obj (.text:strtold)
                  0080bd60    000004c0                     : _scanfi.obj (.text:_sproc_int)
                  0080c220    00000480                     : strtoll.obj (.text:strtoll)
                  0080c6a0    00000460                     : _printfi.obj (.text:_printfi)
                  0080cb00    00000460                     : _printfi.obj (.text:_setfield)
                  0080cf60    00000440     KeyStone_common.obj (.text:Core_MPAX)
                  0080d3a0    00000400     rts6600_elf.lib : strtoull.obj (.text:strtoull)
                  0080d7a0    000003c0                     : strtol.obj (.text:strtol)
                  0080db60    000003a0                     : fputs.obj (.text:fputs)
                  0080df00    00000380                     : fgets.obj (.text:_dofgets)
                  0080e280    00000360     mem_test_DMA_drv.obj (.text)
                  0080e5e0    00000340     rts6600_elf.lib : _scanfi.obj (.text:_sget_conv)
                  0080e920    00000320                     : _printfi.obj (.text:_pproc_fge)
                  0080ec40    00000320                     : strtoul.obj (.text:strtoul)
                  0080ef60    000002e0                     : _printfi.obj (.text:_pproc_fwp)
                  0080f240    000002e0                     : _scanfi.obj (.text:_sproc_float)
                  0080f520    000002a0                     : _printfi.obj (.text:fcvt)
                  0080f7c0    00000280                     : divf.obj (.text:__c6xabi_divf)
                  0080fa40    00000280                     : _printfi.obj (.text:ecvt)
                  0080fcc0    00000280                     : memory.obj (.text:free)
                  0080ff40    00000240                     : imath64.obj (.text:__c6xabi_divull)
                  00810180    00000240                     : _printfi.obj (.text:_pconv_e)
                  008103c0    00000240                     : _printfi.obj (.text:_pproc_diouxp)
                  00810600    00000220                     : _printfi.obj (.text:_pproc_str)
                  00810820    00000220                     : fputc.obj (.text:fputc)
                  00810a40    00000200                     : _printfi.obj (.text:_pconv_g)
                  00810c40    00000200                     : setvbuf.obj (.text:setvbuf)
                  00810e40    000001c0                     : _printfi.obj (.text:_mcpy)
                  00811000    000001c0                     : fopen.obj (.text:_openfile)
                  008111c0    000001a0                     : trgdrv.obj (.text:HOSTrename)
                  00811360    000001a0                     : imath40.obj (.text:__c6xabi_divul)
                  00811500    000001a0                     : _scanfi.obj (.text:_sproc_lb)
                  008116a0    000001a0                     : _scanfi.obj (.text:_sproc_str)
                  00811840    00000180                     : copy_decompress_rle.obj (.text:__TI_decompress_rle_core)
                  008119c0    00000180                     : memory.obj (.text:malloc)
                  00811b40    00000180                     : lowlev.obj (.text:open)
                  00811cc0    00000140                     : sscanf.obj (.text:_chkmbc)
                  00811e00    00000140                     : _printfi.obj (.text:_pproc_fflags)
                  00811f40    00000140                     : lowlev.obj (.text:getdevice)
                  00812080    00000140     mem_test_get_unused_L2_address.obj (.text)
                  008121c0    00000120     rts6600_elf.lib : _bufread.obj (.text:_buff_read)
                  008122e0    00000120                     : fclose.obj (.text:_closefile)
                  00812400    00000120                     : _printfi.obj (.text:_ltostr)
                  00812520    00000120                     : fopen.obj (.text:_search_fp)
                  00812640    00000120                     : _scanfi.obj (.text:_sget_scanset)
                  00812760    00000120                     : fseek.obj (.text:fseek)
                  00812880    00000100                     : trgdrv.obj (.text:HOSTlseek)
                  00812980    00000100                     : autoinit.obj (.text:_auto_init_elf)
                  00812a80    00000100                     : _io_perm.obj (.text:_wrt_ok)
                  00812b80    00000100                     : cpy_tbl.obj (.text:copy_in)
                  00812c80    000000e0                     : trgdrv.obj (.text:HOSTopen)
                  00812d60    000000e0                     : _printfi.obj (.text:_div)
                  00812e40    000000e0                     : atoi.obj (.text:atoi)
                  00812f20    000000e0                     : lowlev.obj (.text:close)
                  00813000    000000e0                     : copy_zero_init.obj (.text:decompress:ZI:__TI_zero_init)
                  008130e0    000000e0                     : ltoa.obj (.text:ltoa)
                  008131c0    000000e0                     : memset.obj (.text:memset)
                  008132a0    000000e0                     : printf.obj (.text:printf)
                  00813380    000000c0                     : trgdrv.obj (.text:HOSTread)
                  00813440    000000c0                     : trgdrv.obj (.text:HOSTunlink)
                  00813500    000000c0                     : trgdrv.obj (.text:HOSTwrite)
                  008135c0    000000c0                     : divu.obj (.text:__divu)
                  00813680    000000c0                     : fflush.obj (.text:_doflush)
                  00813740    000000c0                     : _io_perm.obj (.text:_rd_ok)
                  00813800    000000c0                     : exit.obj (.text:exit)
                  008138c0    000000c0                     : tls.obj (.text:tls:init:__TI_tls_init)
                  00813980    000000a0                     : trgdrv.obj (.text:HOSTclose)
                  00813a20    000000a0                     : remu.obj (.text:__remu)
                  00813ac0    000000a0                     : fopen.obj (.text:_cleanup)
                  00813b60    000000a0                     : _printfi.obj (.text:_ecpy)
                  00813c00    000000a0                     : _printfi.obj (.text:_fcpy)
                  00813ca0    000000a0                     : memory.obj (.text:_minit)
                  00813d40    000000a0                     : _printfi.obj (.text:_pconv_f)
                  00813de0    000000a0                     : lowlev.obj (.text:finddevice)
                  00813e80    000000a0                     : lowlev.obj (.text:lseek)
                  00813f20    000000a0                     : memcpy64.obj (.text:memcpy)
                  00813fc0    000000a0                     : memory.obj (.text:minsert)
                  00814060    000000a0                     : memory.obj (.text:mremove)
                  00814100    000000a0                     : lowlev.obj (.text:read)
                  008141a0    000000a0                     : lowlev.obj (.text:write)
                  00814240    00000080                     : fixdu.obj (.text:__c6xabi_fixdu)
                  008142c0    00000080                     : fixfu.obj (.text:__c6xabi_fixfu)
                  00814340    00000080                     : llshift.obj (.text:__c6xabi_llshl)
                  008143c0    00000080                     : boot.obj (.text:_c_int00)
                  00814440    00000080                     : trgmsg.obj (.text:readmsg)
                  008144c0    00000080                     : lowlev.obj (.text:unlink)
                  00814540    00000060                     : cpp_init.obj (.text:__TI_cpp_init)
                  008145a0    00000060                     : frcmpyd_div.obj (.text:__c6xabi_frcmpyd_div)
                  00814600    00000060                     : llshift.obj (.text:__c6xabi_llshru)
                  00814660    00000060                     : imath64.obj (.text:__c6xabi_remull)
                  008146c0    00000060                     : imath64.obj (.text:_subcull)
                  00814720    00000060                     : fclose.obj (.text:fclose)
                  00814780    00000060                     : fopen.obj (.text:fopen)
                  008147e0    00000060                     : memccpy.obj (.text:memccpy)
                  00814840    00000060                     : sscanf.obj (.text:sscanf)
                  008148a0    00000060                     : lowlev.obj (.text:tabinit)
                  00814900    00000060                     : trgmsg.obj (.text:writemsg)
                  00814960    00000040                     : isinf.obj (.text:__c6xabi_isinf)
                  008149a0    00000040                     : _printfi.obj (.text:__c6xabi_isnan)
                  008149e0    00000040                     : strasg.obj (.text:__strasgi_64plus)
                  00814a20    00000040                     : args_main.obj (.text:_args_main)
                  00814a60    00000040                     : fputs.obj (.text:puts)
                  00814aa0    00000040                     : strlen.obj (.text:strlen)
                  00814ae0    00000020                     : errno.obj (.text:__c6xabi_errno_addr)
                  00814b00    00000020                     : negll.obj (.text:__c6xabi_negll)
                  00814b20    00000020                     : sscanf.obj (.text:_inpchar)
                  00814b40    00000020                     : _lock.obj (.text:_nop)
                  00814b60    00000020                     : printf.obj (.text:_outc)
                  00814b80    00000020                     : printf.obj (.text:_outs)
                  00814ba0    00000020                     : sscanf.obj (.text:_uninpchar)
                  00814bc0    00000020                     : exit.obj (.text:abort)
                  00814be0    00000020                     : copy_decompress_none.obj (.text:decompress:none:__TI_decompress_none)
                  00814c00    00000020                     : copy_decompress_rle.obj (.text:decompress:rle24:__TI_decompress_rle24)
                  00814c20    00000020                     : fgets.obj (.text:fgets)

.switch    0    00814c40    00000028     
                  00814c40    00000028     rts6600_elf.lib : _scanfi.obj (.switch:_sset_arg)

.stack     0    00814c68    00001000     UNINITIALIZED
                  00814c68    00000008     rts6600_elf.lib : boot.obj (.stack)
                  00814c70    00000ff8     --HOLE--

.far       0    00815c68    00008210     
                  00815c68    00008000     mem_test_main.obj (.far) [fill = 0]
                  0081dc68    00000140     rts6600_elf.lib : defs.obj (.far) [fill = 0]
                  0081dda8    00000068     KeyStone_common.obj (.far) [fill = 0]
                  0081de10    00000050     mem_test_main.obj (.far:Core_MPAX)
                  0081de60    00000010     KeyStone_common.obj (.far:Core_MPAX)
                  0081de70    00000008     rts6600_elf.lib : trgdrv.obj (.far) [fill = 0]

.bss       0    0081de78    00000020     UNINITIALIZED
                  0081de78    00000020     mem_test_main.obj (.bss)

.sysmem    0    0081de98    00000800     UNINITIALIZED
                  0081de98    00000008     rts6600_elf.lib : memory.obj (.sysmem)
                  0081dea0    000007f8     --HOLE--

.fardata   0    0081e698    00000484     
                  0081e698    000001e0     rts6600_elf.lib : defs.obj (.fardata:_ftable)
                  0081e878    000000a0                     : lowlev.obj (.fardata:_stream)
                  0081e918    00000078                     : lowlev.obj (.fardata:_device)
                  0081e990    00000040     KeyStone_common.obj (.fardata:gstruMpuAddrRange)
                  0081e9d0    00000028     KeyStone_common.obj (.fardata:gEDMA_TC_Regs)
                  0081e9f8    00000024     KeyStone_common.obj (.fardata:internal_exception_str)
                  0081ea1c    00000004     rts6600_elf.lib : defs.obj (.fardata)
                  0081ea20    00000024     KeyStone_common.obj (.fardata:timerRegs)
                  0081ea44    00000004     rts6600_elf.lib : errno.obj (.fardata)
                  0081ea48    00000020     KeyStone_common.obj (.fardata:MPU_Regs)
                  0081ea68    00000020     KeyStone_common.obj (.fardata:bus_err_stat_str)
                  0081ea88    00000020     KeyStone_common.obj (.fardata:gCIC_EXC_EN_MASK)
                  0081eaa8    00000020     mem_test_DSP_core.obj (.fardata:ulDataPatternTable)
                  0081eac8    00000018     KeyStone_common.obj (.fardata:Peri_MPU_err_type_str)
                  0081eae0    0000000c     KeyStone_common.obj (.fardata:gEDMACCRegs)
                  0081eaec    0000000c     rts6600_elf.lib : exit.obj (.fardata)
                  0081eaf8    0000000c                     : memory.obj (.fardata)
                  0081eb04    00000004                     : fopen.obj (.fardata)
                  0081eb08    00000008     KeyStone_common.obj (.fardata:Ns_str)
                  0081eb10    00000008     rts6600_elf.lib : _lock.obj (.fardata)
                  0081eb18    00000004                     : lowlev.obj (.fardata)

.const     0    0081eb20    0000225e     
                  0081eb20    00001628     KeyStone_common.obj (.const:.string)
                  00820148    000003bc     mem_test_DMA.obj (.const:.string)
                  00820504    00000284     mem_test_main.obj (.const:.string)
                  00820788    00000274     mem_test_DSP_core.obj (.const:.string)
                  008209fc    00000002     rts6600_elf.lib : fputs.obj (.const:.string)
                  008209fe    00000002     --HOLE-- [fill = 0]
                  00820a00    00000101                     : ctype.obj (.const:.string:_ctypes_)
                  00820b01    00000003     --HOLE-- [fill = 0]
                  00820b04    000000c4     KeyStone_DDR_Init.obj (.const:.string)
                  00820bc8    00000050     mem_test_get_unused_L2_address.obj (.const:.string)
                  00820c18    00000050     rts6600_elf.lib : strtod.obj (.const:digits)
                  00820c68    00000050                     : strtold.obj (.const:digits)
                  00820cb8    00000048                     : strtod.obj (.const:powerof10)
                  00820d00    00000048                     : strtold.obj (.const:powerof10)
                  00820d48    00000023                     : _printfi.obj (.const:.string)
                  00820d6b    00000005     --HOLE-- [fill = 0]
                  00820d70    00000007                     : _scanfi.obj (.const:.string:flit$1)
                  00820d77    00000001     --HOLE-- [fill = 0]
                  00820d78    00000006                     : _scanfi.obj (.const:.string:barr$2)

.neardata 
*          0    00820d80    000000c4     
                  00820d80    000000b8     KeyStone_common.obj (.neardata)
                  00820e38    00000008     mem_test_main.obj (.neardata)
                  00820e40    00000004     mem_test_DMA.obj (.neardata)

.rodata    0    00820e44    00000000     UNINITIALIZED

.cinit     0    00820e44    000002e8     
                  00820e44    00000199     (.cinit..fardata.load) [load image, compression = rle]
                  00820fdd    00000003     --HOLE-- [fill = 0]
                  00820fe0    000000bc     (.cinit..neardata.load) [load image, compression = rle]
                  0082109c    0000005b     (.cinit..far.load) [load image, compression = rle]
                  008210f7    00000001     --HOLE-- [fill = 0]
                  008210f8    0000000c     (__TI_handler_table)
                  00821104    00000008     (.cinit..bss.load) [load image, compression = zero_init]
                  0082110c    00000020     (__TI_cinit_table)

.cio       0    0082112c    00000120     UNINITIALIZED
                  0082112c    00000120     rts6600_elf.lib : trgmsg.obj (.cio)


LINKER GENERATED COPY TABLES

__TI_cinit_table @ 0082110c records: 4, size/record: 8, table size: 32
	.fardata: load addr=00820e44, load size=00000199 bytes, run addr=0081e698, run size=00000484 bytes, compression=rle
	.neardata: load addr=00820fe0, load size=000000bc bytes, run addr=00820d80, run size=000000c4 bytes, compression=rle
	.far: load addr=0082109c, load size=0000005b bytes, run addr=00815c68, run size=00008210 bytes, compression=rle
	.bss: load addr=00821104, load size=00000008 bytes, run addr=0081de78, run size=00000020 bytes, compression=zero_init


LINKER GENERATED HANDLER TABLE

__TI_handler_table @ 008210f8 records: 3, size/record: 4, table size: 12
	index: 0, handler: __TI_decompress_rle24
	index: 1, handler: __TI_decompress_none
	index: 2, handler: __TI_zero_init


GLOBAL SYMBOLS: SORTED ALPHABETICALLY BY Name 

address    name
--------   ----
00809668   Bus_Bit_Walking
00804130   Bus_error_handler
00814bc0   C$$EXIT
00814958   C$$IO$$
0080644c   C6670_EVM_DDR_Init
00805590   C6678_EVM_DDR_Init
00820d84   CGEM_regs
00820da8   CIC_Regs
0080718c   DDR_Address_Test
00807290   DDR_Fill_Test
00820d9c   DDR_Regs
008082a8   DMA_MEM_AddrTest
008080a0   DMA_MEM_FillTest
00820e14   DSP_Core_Clock_KHz
008098ac   DSP_core_MEM_Test
00805c28   Dual_Nyquist_EVM_DDR_Init
00801cd4   EDMA_CC_error_handler
0080e4c4   EDMA_Copy
008084e4   EDMA_MEM_Bit_Walking
0080876c   EDMA_MEM_Test
00801ee4   EDMA_TC_error_handler
00801a28   EDMA_copy
00802014   EDMA_error_handler
0080e280   EDMA_init_for_mem_test
00801968   EDMA_wait
00804bd0   EXC_NMI
00804b10   EXC_internal
00804be8   EXC_swgen
0080a1a0   Exception_service_routine
00813980   HOSTclose
00812880   HOSTlseek
00812c80   HOSTopen
00813380   HOSTread
008111c0   HOSTrename
00813440   HOSTunlink
00813500   HOSTwrite
0080864c   IDMA_MEM_Bit_Walking
00808954   IDMA_MEM_Test
00801c34   IDMA_copy
00801c08   IDMA_wait
0080420c   KeyStone_CIC_EXC_handler
00803acc   KeyStone_CIC_exception_events_mapping
00802524   KeyStone_CorePac_AID_map
0080526c   KeyStone_DDR_ECC_INT_enable
00805290   KeyStone_DDR_ECC_init
00804f28   KeyStone_DDR_PLL_init
00805484   KeyStone_DDR_clock_phase_init
008050d4   KeyStone_DDR_full_leveling
00807388   KeyStone_DDR_init
00805544   KeyStone_DDR_latch_leveling_configuration
0080516c   KeyStone_DDR_read_incremental_leveling
0080464c   KeyStone_EXC_external
00803f24   KeyStone_Exception_cfg
00807844   KeyStone_LL2_memory_EDMA_test
00807694   KeyStone_LL2_memory_test
0080d0f0   KeyStone_MPAX_seg_setup
00802d30   KeyStone_MPU_MPPA_modify
00802e28   KeyStone_MPU_interrupts_enable
00802aac   KeyStone_MPU_range_setup
00802b2c   KeyStone_MPU_setup
008027e8   KeyStone_MSMC_MP_interrupt_en
00802968   KeyStone_MSMC_protection_exception_handler
008025ac   KeyStone_PrivID_Remap
00802708   KeyStone_SES_MPAX_setup
008031e0   KeyStone_SL2_EDC_enable
008037f4   KeyStone_SL2_EDC_handler
008032a0   KeyStone_SL2_EDC_interrupt_en
008079f0   KeyStone_SL2_memory_EDMA_test
00807798   KeyStone_SL2_memory_test
00802628   KeyStone_SMS_MPAX_setup
0080d294   KeyStone_XMC_MPAX_setup
0080130c   KeyStone_disable_PSC_Power_Domain
008012b4   KeyStone_disable_PSC_module
00801250   KeyStone_enable_PSC_module
00807c84   KeyStone_external_memory_EDMA_test
00807c30   KeyStone_external_memory_test
008008ec   KeyStone_main_PLL_init
00807b04   KeyStone_other_L1_memory_EDMA_test
00807914   KeyStone_other_L2_memory_EDMA_test
008076e8   KeyStone_other_L2_memory_test
00803100   KeyStone_peripherals_MPU_excepiton_handler
00803004   KeyStone_peripherals_MPU_fault_status
00804c00   KeyStone_print_device_info
008077ec   KeyStone_remapped_SL2_memory_test
00802250   L1D_memory_protection_cfg
0080344c   L1P_EDC_setup
008036d0   L1P_ED_handler
008021c0   L1P_memory_protection_cfg
00802118   L1_MPPA_setup
008022e4   L1_cache_protection
00807a78   LL1_memory_IDMA_test
00820e24   LL2_EDC_DMA_err_str
00820e28   LL2_EDC_L1D_err_str
00820e2c   LL2_EDC_L1P_err_str
008034d0   LL2_EDC_handler
008033b4   LL2_EDC_scrub
008032f4   LL2_EDC_setup
00820e20   LL2_EDC_victim_err_str
008022f4   LL2_MPPA_setup
00802390   LL2_Memory_Protection_cfg
00809554   MEM_AddrTest
008097ac   MEM_Bit_Walking
00809440   MEM_FillTest
00820e04   MPU0_Regs
00820e08   MPU1_Regs
00820e0c   MPU2_Regs
00820e10   MPU3_Regs
0081ea48   MPU_Regs
0080a54c   Nested_Exception_service_routine
0081eb08   Ns_str
0081eac8   Peri_MPU_err_type_str
00800f04   Reset_Timer
0080120c   Service_Watchdog
00806ac0   TCI6614_EVM_DDR_Init
00820e40   TC_channel
00802a60   TN_MPU5_constant
00800da8   TSC_delay_ms
00800e60   TSC_delay_us
00800d94   TSC_init
00800f50   Timer64_Init
0081de10   XMC_MPAX_cfg_table
00820d80   XMC_regs
0082112c   __CIOBUF_
0082110c   __TI_CINIT_Base
0082112c   __TI_CINIT_Limit
008210f8   __TI_Handler_Table_Base
00821104   __TI_Handler_Table_Limit
UNDEFED    __TI_INITARRAY_Base
UNDEFED    __TI_INITARRAY_Limit
00815c68   __TI_STACK_END
00001000   __TI_STACK_SIZE
0081de78   __TI_STATIC_BASE
00000800   __TI_SYSMEM_SIZE
UNDEFED    __TI_TLS_INIT_Base
UNDEFED    __TI_TLS_INIT_Limit
00000001   __TI_args_main
00814540   __TI_cpp_init
00814be0   __TI_decompress_none
00814c00   __TI_decompress_rle24
0081eaf4   __TI_enable_exit_profile_output
ffffffff   __TI_pprof_out_hndl
ffffffff   __TI_prof_data_size
ffffffff   __TI_prof_data_start
008138c0   __TI_tls_init
00813000   __TI_zero_init
ffffffff   __binit__
0080a7a0   __c6xabi_divd
0080f7c0   __c6xabi_divf
008135c0   __c6xabi_divu
00811360   __c6xabi_divul
0080ff40   __c6xabi_divull
00814ae0   __c6xabi_errno_addr
00814240   __c6xabi_fixdu
008142c0   __c6xabi_fixfu
008145a0   __c6xabi_frcmpyd_div
00814960   __c6xabi_isinf
00814340   __c6xabi_llshl
00814600   __c6xabi_llshru
00814b00   __c6xabi_negll
00813a20   __c6xabi_remu
00814660   __c6xabi_remull
008149e0   __c6xabi_strasgi_64plus
ffffffff   __c_args__
008135c0   __divu
0081ea44   __errno
00813a20   __remu
008149e0   __strasgi_64plus
00814a20   _args_main
00812980   _auto_init_elf
008121c0   _buff_read
008143c0   _c_int00
00813ac0   _cleanup
0081eaec   _cleanup_ptr
008122e0   _closefile
00820a00   _ctypes_
00813680   _doflush
0081eaf0   _dtors_ptr
0081ea1c   _ft_end
0081e698   _ftable
0081eb10   _lock
00813ca0   _minit
00814b40   _nop
0080c6a0   _printfi
00813740   _rd_ok
00808b00   _scanfi
00814c68   _stack
008146c0   _subcull
0081de98   _sys_memory
0081dc68   _tmpnams
0081eb14   _unlock
00812a80   _wrt_ok
00814bc0   abort
00812e40   atoi
ffffffff   binit
00820d88   boot_cfg_regs
0081ea68   bus_err_stat_str
00800d40   calc_cycle_measure_overhead
00812f20   close
00812b80   copy_in
00820da0   cpIntc0Regs
00820da4   cpIntc1Regs
00820e18   cycle_measure_overhead
00815c68   dma_buf
00801410   edma_Init
008013bc   edma_TC_priority_cfg
00801358   edma_channel_TC_cfg
0081ea44   errno
0081dda8   exception_record
00813800   exit
00814720   fclose
00814c20   fgets
00814780   fopen
00810820   fputc
0080db60   fputs
0080fcc0   free
00812760   fseek
0081ea88   gCIC_EXC_EN_MASK
00820e34   gCIC_EXC_out_num
00820dac   gEDMACC0Regs
00820db0   gEDMACC1Regs
00820db4   gEDMACC2Regs
0081eae0   gEDMACCRegs
00820db8   gEDMA_TC_0_0_Regs
00820dbc   gEDMA_TC_0_1_Regs
00820dc0   gEDMA_TC_1_0_Regs
00820dc4   gEDMA_TC_1_1_Regs
00820dc8   gEDMA_TC_1_2_Regs
00820dcc   gEDMA_TC_1_3_Regs
00820dd0   gEDMA_TC_2_0_Regs
00820dd4   gEDMA_TC_2_1_Regs
00820dd8   gEDMA_TC_2_2_Regs
00820ddc   gEDMA_TC_2_3_Regs
0081e9d0   gEDMA_TC_Regs
00812080   get_unused_L2_address
00820d98   gpioRegs
0081e990   gstruMpuAddrRange
00820e30   guwIntcCICExcEvtIdx
00820e38   iFailedTimes
00820e3c   iPassedTimes
0081e9f8   internal_exception_str
0080cf60   lock_mem_prot_regs
00813e80   lseek
008130e0   ltoa
00807d10   main
008119c0   malloc
0081de60   mem_prot_key
008147e0   memccpy
00813f20   memcpy
00802850   memory_protection_exception_handler
008131c0   memset
00820d94   msmcRegs
0081de8c   number_of_cores
00811b40   open
00807644   pass_fail_count
00820d8c   pllc_regs
008132a0   printf
00820d90   pscRegs
00814a60   puts
00814100   read
00814440   readmsg
008144c0   remove
00810c40   setvbuf
00814840   sscanf
00814aa0   strlen
0080b320   strtod
0080d7a0   strtol
0080b840   strtold
0080c220   strtoll
0080ec40   strtoul
0080d3a0   strtoull
00820de0   timer0Regs
00820de4   timer1Regs
00820de8   timer2Regs
00820dec   timer3Regs
00820df0   timer4Regs
00820df4   timer5Regs
00820df8   timer6Regs
00820dfc   timer7Regs
00820e00   timer8Regs
0081ea20   timerRegs
0081de94   tsch
0081de90   tscl
0081de88   uiDDREndAddress
0081de7c   uiLL2EndAddress
0081de78   uiLL2StartAddress
00820e1c   uiLL2_scrub_addr
0081de84   uiRemappedSL2EndAddress
0081de80   uiSL2EndAddress
0081eaa8   ulDataPatternTable
008144c0   unlink
0080d028   unlock_mem_prot_regs
008141a0   write
00814900   writemsg


GLOBAL SYMBOLS: SORTED BY Symbol Address 

address    name
--------   ----
00000001   __TI_args_main
00000800   __TI_SYSMEM_SIZE
00001000   __TI_STACK_SIZE
008008ec   KeyStone_main_PLL_init
00800d40   calc_cycle_measure_overhead
00800d94   TSC_init
00800da8   TSC_delay_ms
00800e60   TSC_delay_us
00800f04   Reset_Timer
00800f50   Timer64_Init
0080120c   Service_Watchdog
00801250   KeyStone_enable_PSC_module
008012b4   KeyStone_disable_PSC_module
0080130c   KeyStone_disable_PSC_Power_Domain
00801358   edma_channel_TC_cfg
008013bc   edma_TC_priority_cfg
00801410   edma_Init
00801968   EDMA_wait
00801a28   EDMA_copy
00801c08   IDMA_wait
00801c34   IDMA_copy
00801cd4   EDMA_CC_error_handler
00801ee4   EDMA_TC_error_handler
00802014   EDMA_error_handler
00802118   L1_MPPA_setup
008021c0   L1P_memory_protection_cfg
00802250   L1D_memory_protection_cfg
008022e4   L1_cache_protection
008022f4   LL2_MPPA_setup
00802390   LL2_Memory_Protection_cfg
00802524   KeyStone_CorePac_AID_map
008025ac   KeyStone_PrivID_Remap
00802628   KeyStone_SMS_MPAX_setup
00802708   KeyStone_SES_MPAX_setup
008027e8   KeyStone_MSMC_MP_interrupt_en
00802850   memory_protection_exception_handler
00802968   KeyStone_MSMC_protection_exception_handler
00802a60   TN_MPU5_constant
00802aac   KeyStone_MPU_range_setup
00802b2c   KeyStone_MPU_setup
00802d30   KeyStone_MPU_MPPA_modify
00802e28   KeyStone_MPU_interrupts_enable
00803004   KeyStone_peripherals_MPU_fault_status
00803100   KeyStone_peripherals_MPU_excepiton_handler
008031e0   KeyStone_SL2_EDC_enable
008032a0   KeyStone_SL2_EDC_interrupt_en
008032f4   LL2_EDC_setup
008033b4   LL2_EDC_scrub
0080344c   L1P_EDC_setup
008034d0   LL2_EDC_handler
008036d0   L1P_ED_handler
008037f4   KeyStone_SL2_EDC_handler
00803acc   KeyStone_CIC_exception_events_mapping
00803f24   KeyStone_Exception_cfg
00804130   Bus_error_handler
0080420c   KeyStone_CIC_EXC_handler
0080464c   KeyStone_EXC_external
00804b10   EXC_internal
00804bd0   EXC_NMI
00804be8   EXC_swgen
00804c00   KeyStone_print_device_info
00804f28   KeyStone_DDR_PLL_init
008050d4   KeyStone_DDR_full_leveling
0080516c   KeyStone_DDR_read_incremental_leveling
0080526c   KeyStone_DDR_ECC_INT_enable
00805290   KeyStone_DDR_ECC_init
00805484   KeyStone_DDR_clock_phase_init
00805544   KeyStone_DDR_latch_leveling_configuration
00805590   C6678_EVM_DDR_Init
00805c28   Dual_Nyquist_EVM_DDR_Init
0080644c   C6670_EVM_DDR_Init
00806ac0   TCI6614_EVM_DDR_Init
0080718c   DDR_Address_Test
00807290   DDR_Fill_Test
00807388   KeyStone_DDR_init
00807644   pass_fail_count
00807694   KeyStone_LL2_memory_test
008076e8   KeyStone_other_L2_memory_test
00807798   KeyStone_SL2_memory_test
008077ec   KeyStone_remapped_SL2_memory_test
00807844   KeyStone_LL2_memory_EDMA_test
00807914   KeyStone_other_L2_memory_EDMA_test
008079f0   KeyStone_SL2_memory_EDMA_test
00807a78   LL1_memory_IDMA_test
00807b04   KeyStone_other_L1_memory_EDMA_test
00807c30   KeyStone_external_memory_test
00807c84   KeyStone_external_memory_EDMA_test
00807d10   main
008080a0   DMA_MEM_FillTest
008082a8   DMA_MEM_AddrTest
008084e4   EDMA_MEM_Bit_Walking
0080864c   IDMA_MEM_Bit_Walking
0080876c   EDMA_MEM_Test
00808954   IDMA_MEM_Test
00808b00   _scanfi
00809440   MEM_FillTest
00809554   MEM_AddrTest
00809668   Bus_Bit_Walking
008097ac   MEM_Bit_Walking
008098ac   DSP_core_MEM_Test
0080a1a0   Exception_service_routine
0080a54c   Nested_Exception_service_routine
0080a7a0   __c6xabi_divd
0080b320   strtod
0080b840   strtold
0080c220   strtoll
0080c6a0   _printfi
0080cf60   lock_mem_prot_regs
0080d028   unlock_mem_prot_regs
0080d0f0   KeyStone_MPAX_seg_setup
0080d294   KeyStone_XMC_MPAX_setup
0080d3a0   strtoull
0080d7a0   strtol
0080db60   fputs
0080e280   EDMA_init_for_mem_test
0080e4c4   EDMA_Copy
0080ec40   strtoul
0080f7c0   __c6xabi_divf
0080fcc0   free
0080ff40   __c6xabi_divull
00810820   fputc
00810c40   setvbuf
008111c0   HOSTrename
00811360   __c6xabi_divul
008119c0   malloc
00811b40   open
00812080   get_unused_L2_address
008121c0   _buff_read
008122e0   _closefile
00812760   fseek
00812880   HOSTlseek
00812980   _auto_init_elf
00812a80   _wrt_ok
00812b80   copy_in
00812c80   HOSTopen
00812e40   atoi
00812f20   close
00813000   __TI_zero_init
008130e0   ltoa
008131c0   memset
008132a0   printf
00813380   HOSTread
00813440   HOSTunlink
00813500   HOSTwrite
008135c0   __c6xabi_divu
008135c0   __divu
00813680   _doflush
00813740   _rd_ok
00813800   exit
008138c0   __TI_tls_init
00813980   HOSTclose
00813a20   __c6xabi_remu
00813a20   __remu
00813ac0   _cleanup
00813ca0   _minit
00813e80   lseek
00813f20   memcpy
00814100   read
008141a0   write
00814240   __c6xabi_fixdu
008142c0   __c6xabi_fixfu
00814340   __c6xabi_llshl
008143c0   _c_int00
00814440   readmsg
008144c0   remove
008144c0   unlink
00814540   __TI_cpp_init
008145a0   __c6xabi_frcmpyd_div
00814600   __c6xabi_llshru
00814660   __c6xabi_remull
008146c0   _subcull
00814720   fclose
00814780   fopen
008147e0   memccpy
00814840   sscanf
00814900   writemsg
00814958   C$$IO$$
00814960   __c6xabi_isinf
008149e0   __c6xabi_strasgi_64plus
008149e0   __strasgi_64plus
00814a20   _args_main
00814a60   puts
00814aa0   strlen
00814ae0   __c6xabi_errno_addr
00814b00   __c6xabi_negll
00814b40   _nop
00814bc0   C$$EXIT
00814bc0   abort
00814be0   __TI_decompress_none
00814c00   __TI_decompress_rle24
00814c20   fgets
00814c68   _stack
00815c68   __TI_STACK_END
00815c68   dma_buf
0081dc68   _tmpnams
0081dda8   exception_record
0081de10   XMC_MPAX_cfg_table
0081de60   mem_prot_key
0081de78   __TI_STATIC_BASE
0081de78   uiLL2StartAddress
0081de7c   uiLL2EndAddress
0081de80   uiSL2EndAddress
0081de84   uiRemappedSL2EndAddress
0081de88   uiDDREndAddress
0081de8c   number_of_cores
0081de90   tscl
0081de94   tsch
0081de98   _sys_memory
0081e698   _ftable
0081e990   gstruMpuAddrRange
0081e9d0   gEDMA_TC_Regs
0081e9f8   internal_exception_str
0081ea1c   _ft_end
0081ea20   timerRegs
0081ea44   __errno
0081ea44   errno
0081ea48   MPU_Regs
0081ea68   bus_err_stat_str
0081ea88   gCIC_EXC_EN_MASK
0081eaa8   ulDataPatternTable
0081eac8   Peri_MPU_err_type_str
0081eae0   gEDMACCRegs
0081eaec   _cleanup_ptr
0081eaf0   _dtors_ptr
0081eaf4   __TI_enable_exit_profile_output
0081eb08   Ns_str
0081eb10   _lock
0081eb14   _unlock
00820a00   _ctypes_
00820d80   XMC_regs
00820d84   CGEM_regs
00820d88   boot_cfg_regs
00820d8c   pllc_regs
00820d90   pscRegs
00820d94   msmcRegs
00820d98   gpioRegs
00820d9c   DDR_Regs
00820da0   cpIntc0Regs
00820da4   cpIntc1Regs
00820da8   CIC_Regs
00820dac   gEDMACC0Regs
00820db0   gEDMACC1Regs
00820db4   gEDMACC2Regs
00820db8   gEDMA_TC_0_0_Regs
00820dbc   gEDMA_TC_0_1_Regs
00820dc0   gEDMA_TC_1_0_Regs
00820dc4   gEDMA_TC_1_1_Regs
00820dc8   gEDMA_TC_1_2_Regs
00820dcc   gEDMA_TC_1_3_Regs
00820dd0   gEDMA_TC_2_0_Regs
00820dd4   gEDMA_TC_2_1_Regs
00820dd8   gEDMA_TC_2_2_Regs
00820ddc   gEDMA_TC_2_3_Regs
00820de0   timer0Regs
00820de4   timer1Regs
00820de8   timer2Regs
00820dec   timer3Regs
00820df0   timer4Regs
00820df4   timer5Regs
00820df8   timer6Regs
00820dfc   timer7Regs
00820e00   timer8Regs
00820e04   MPU0_Regs
00820e08   MPU1_Regs
00820e0c   MPU2_Regs
00820e10   MPU3_Regs
00820e14   DSP_Core_Clock_KHz
00820e18   cycle_measure_overhead
00820e1c   uiLL2_scrub_addr
00820e20   LL2_EDC_victim_err_str
00820e24   LL2_EDC_DMA_err_str
00820e28   LL2_EDC_L1D_err_str
00820e2c   LL2_EDC_L1P_err_str
00820e30   guwIntcCICExcEvtIdx
00820e34   gCIC_EXC_out_num
00820e38   iFailedTimes
00820e3c   iPassedTimes
00820e40   TC_channel
008210f8   __TI_Handler_Table_Base
00821104   __TI_Handler_Table_Limit
0082110c   __TI_CINIT_Base
0082112c   __CIOBUF_
0082112c   __TI_CINIT_Limit
ffffffff   __TI_pprof_out_hndl
ffffffff   __TI_prof_data_size
ffffffff   __TI_prof_data_start
ffffffff   __binit__
ffffffff   __c_args__
ffffffff   binit
UNDEFED    __TI_INITARRAY_Base
UNDEFED    __TI_INITARRAY_Limit
UNDEFED    __TI_TLS_INIT_Base
UNDEFED    __TI_TLS_INIT_Limit

[293 symbols]
